:1000000000308A00BB2F00000A108A100A118207F4
:1000100000346634FF34FF347E343C34183400340A
:10002000003418343C347E347E343C34183400348C
:10003000003418347E347E341834183418340034C4
:1000400000347E347E347E347E347E347E3400341C
:100050000034423418340034423424341834003428
:100060000034423418340034183424344234003418
:1000700018343C347E341834183418341834183496
:10008000183418341834183418347E343C34183486
:100090000A108A100A114F3E03188A0A820000349F
:1000A0000034003400340034003400340034203490
:1000B00020342034203420340034203400345034B0
:1000C00050345034003400340034003400345034A0
:1000D0005034F83450345034F834503450342034E0
:1000E0007834A03470342834F03420342034003490
:1000F000C034C834103420344034983418340034B8
:1001000060349034A0344034A8349034683460347F
:1001100020344034003400340034003400341034CF
:10012000203440344034403440342034103440349F
:10013000203410341034103410342034403400345F
:100140002034A8347034A83420340034003400340F
:1001500020342034F8342034203400340034003487
:10016000003400340034003460342034403400342F
:1001700000340034F83400340034003400340034E7
:10018000003400340034003400346034603400340F
:100190000834103420344034803400340034703457
:1001A00088349834A834C83488348834703420347F
:1001B00060342034203420342034203470347034BF
:1001C000883408341034203440348034F834F8341F
:1001D0001034203410340834083488347034103427
:1001E0003034503490349034F83410341034F834BF
:1001F00080348034F0340834083488347034303437
:1002000040348034F0348834883488347034F8349E
:100210000834103420344034403440344034703496
:100220008834883470348834883488347034703436
:1002300088348834883478340834103460340A14AC
:100240008A100A1182077034883408346834A8345C
:10025000A834A83470347034883488348834F8343E
:10026000883488348834F03488348834F0348834DE
:1002700088348834F0347034883480348034803466
:10028000803488347034E03490348834883488344E
:1002900088349034E034F83480348034F834803456
:1002A00080348034F834F83480348034F03480344E
:1002B000803480348034703488348034F834883426
:1002C000883488347834883488348834F8348834EE
:1002D00088348834883470342034203420342034F6
:1002E0002034203470343834103410341034103446
:1002F00010349034603488349034A034C034A03446
:10030000903488348834803480348034803480342D
:1003100080348034F8348834D834A834A83488340D
:1003200088348834883488348834C834A83498347D
:1003300088348834883470348834883488348834F5
:10034000883488347034F034883488348834F03415
:1003500080348034803470348834883488348834ED
:10036000A83490346834F03488348834F034C0349D
:10037000A034903488347834803480347034083435
:1003800008340834F034F834203420342034203455
:1003900020342034203488348834883488348834B5
:1003A0008834883470348834883488348834883485
:1003B0008834503420348834883488348834A834DD
:1003C000A834A8345034883488345034203450341D
:1003D00088348834883488348834883450342034DD
:1003E000203420342034F83408341034203440349D
:1003F00080348034F83459083F3C03181F2A5908C8
:100400005A3C031C1F2A40305902F700770DD900CF
:10041000D90DD90DF830D905DA015A08073C031C6B
:100420001B2A28305A0784005908D90A1F21F800CE
:100430008000DA0A0D2A0530F800692A692A59086D
:100440001F3C0318432A5908393C031C432A203017
:100450005902F700770DD900D90DD90DF830D9051B
:10046000DA015A08073C031C3F2A28305A07840047
:100470005908D90A4820F8008000DA0A312A0530E4
:10048000F800692A692A59080F3C0318672A590895
:10049000173C031C672A10305902F700770DD9006A
:1004A000D90DD90DF830D905DA015A08073C031CDB
:1004B000632A28305A0784005908D90A0420F80012
:1004C0008000DA0A552A0830F800692A692A0030C3
:1004D000F8000034D9015908073C031C7D2A20305C
:1004E0005907DA002830590784000008DB005A0851
:1004F00084005B088000D90A6B2A0034DD080319E8
:10050000FB2ADF015F08073C031CF92A5F1C8D2AC8
:100510008316051183120515912A8316051183127E
:100520000511DF1C982A83168511831285159C2AD4
:1005300083168511831285115F1DA32A8316051268
:1005400083120516A72A831605128312051220307E
:100550005F0784000008E000E100831605108312A5
:1005600005108316851083128510E2016208073C8E
:10057000031CD12A611CC12A831685138312851797
:10058000C52A83168513831285130310E10C831685
:100590000510831205148316051083120510E20A54
:1005A000B62A83168510831285148316851083124C
:1005B000851083160513831205133C30DE00DE031D
:1005C0000319F32A8316061400308312061801302B
:1005D000003A031DF22A8316051383120517013012
:1005E000F800FD2ADF2A8316051383120517DF0A98
:1005F000822ADD037E2A0030F8000034D901590830
:10060000073C031C092B2830590784008001D90AB4
:10061000FF2A0034831605138312051760308316F2
:100620008F000F080439043C031D112B1130831275
:10063000D900FB216A226430DD007E22FE226A227C
:10064000831681138312C52F831606168312DD01CC
:10065000061ADD0A03105D0DDE00831686160030D3
:100660008312861A01305E04DD0003105D0DDE008A
:100670008316061700308312061B01305E04DD006E
:1006800003105D0DDE008316861700308312861B73
:1006900001305E04DD005D08FF3A0F39F8000034D8
:1006A000831606158312DD010619DD0A03105D0DA0
:1006B000DE008316851600308312851A01305E0431
:1006C000DD0003105D0DDE008316861500308312F9
:1006D000861901305E04DD0003105D0DDE00831617
:1006E000861400308312861801305E04DD005D0838
:1006F000F8000034D9015908073C031C922B28301C
:100700005907DA00283059078400000CF700F70C6D
:100710003F30F7057708DC005A0884005C08800049
:10072000D90A7B2B00340730D9005908003C031844
:10073000A82B20305907DA0001305902203E8400EE
:100740000008DC005A0884005C088000D903952B5F
:100750000034242378080339DC00DC08031DB42BA3
:100760001130F800C42BC42B5C0BBA2B0E30F800F0
:10077000C42BC42B5C08023C031DC22B0B30F800B9
:10078000C42BC42B0830F80000349323A001A92304
:100790007808D900DD007E220830D8005808003CD7
:1007A0000318E02B932301305802283E84000008F0
:1007B000A000A9237808D900DD007E22D803CE2B23
:1007C0000034D9015908063C031CF52B2030590789
:1007D000DA0001305907203E84000008DC005A0886
:1007E00084005C088000D90AE22B0034E123A701D1
:1007F000A9237808D900DD007E22D8015808073CDB
:10080000031C0F2CE1232830580784000008A700A0
:10081000A9237808D900DD007E22D80AFE2B0034F7
:10082000FF30D50050237808D4005508540203192E
:10083000612C1930DD007E22502378085402031DFC
:100840005F2C5408D600D608031D292C4730D6004B
:10085000502C56080B3C031D302C4130D600502C38
:1008600056080C3C031D372C4230D600502C56083D
:100870000D3C031D3E2C4330D600502C56080E3C38
:10088000031D452C4430D600502C56080F3C031D48
:100890004C2C2030D600502C013056023038D60077
:1008A0005608D900FB217A23550F582C6A225F2C59
:1008B0005408550203185E2CC5235F2CF6235408F8
:1008C000D5000530DD007E22122CCD2F0830F70038
:1008D00083160614831206186B2CD801F7177E2C8A
:1008E000F7137E2C031006180314D80C77177E2CF0
:1008F0007713F70B722C5808F8008B2C8430F71BF9
:100900002430F800F80B822C00000000F71B702C3C
:10091000771B782C722C8F2CD601D701662C780887
:10092000D50055083A3C031D992CD6010130D7005B
:10093000B12C55080D3C031DA42C30305607840003
:1009400055088000B22CB12CD7080319B12C5608D9
:10095000213C031CB12C5608D60A303E84005508B1
:1009600080008E2C003450237808DB005B085A028C
:10097000031DD12CDC015C08213C031CCE2C303043
:100980005C07DD0001305C07303E84000008DF00BA
:100990005D0884005F088000DC0ABB2C0030F80092
:1009A000D32C0130F8000034DB015B085902031C32
:1009B000FE2CDA015A08073C031CF72C20305A079A
:1009C00084000310000D800028305A078400801F27
:1009D000EF2C20305A0784000008013880002830AE
:1009E0005A0784000310000D8000DA0ADA2CA923CC
:1009F0007808DC00DD007E22DB0AD52C00345A08A2
:100A00000D3C031D062D0D30F800152D5A082F3C06
:100A10000318132D5A08373C031C132D20305A029B
:100A2000F800152D152D0030F8000034F701F801FD
:100A30005B0803105C18F707F70CF80CDC18F707D5
:100A4000F70CF80C5C19F707F70CF80CDC19F70732
:100A5000F70CF80C5C1AF707F70CF80CDC1AF70720
:100A6000F70CF80C5C1BF707F70CF80CDC1BF7070E
:100A7000F70CF80C022ED6013008603C0318472D05
:100A800030087A3C031C472D3008DF39482D3008E8
:100A9000D50055082F3C0318582D5508393C031C28
:100AA000582D55080F39D800DA00B3247808D6003D
:100AB0005508403C0318682D5508463C031C682D1A
:100AC00055080F39093ED900DA00B3247808D6005A
:100AD000560B6B2DE42E3008603C0318762D300841
:100AE0007A3C031C762D3008DF39772D3008D5008D
:100AF0005508543C031DC42D0130D6002030D900C8
:100B0000FB217808D800D900D4245608D60A303EF4
:100B100084000008D900603C0318952D59087A3CE0
:100B2000031C952D5908DF39962D5908D500550815
:100B30005C3C031DA52D5608D60A303E84000008F3
:100B4000D900DA00FF247808D50055080D3C031DB4
:100B5000B82D2030D900FB217808D800D900D42442
:100B60002030D900FB217808D800D900D424E42E05
:100B7000D5080319C22D5508D900FB217808D800E3
:100B8000D900D424852DE42E5508583C031DE42EAD
:100B90003308603C0318D32D33087A3C031CD32D53
:100BA0003308DF39D42D3308D70057085C3C031DC8
:100BB000DE2D3408DA00FF247808D7005708D90062
:100BC000FB217808053C031DE62D7A233108603CA3
:100BD0000318F12D31087A3C031CF12D3108DF395F
:100BE000F22D3108D5003208303C031DFA2D0130BA
:100BF000D600042E32080F39013EDA00DB0019302E
:100C0000DC00162D7808D60043305502ED3E03185F
:100C1000E42E133EE52EF6235608DD007E22E42E58
:100C2000C5235608DD007E22E42EA9237808DA00C9
:100C3000DD007E22D9015908073C031C442ED8014F
:100C40005808073C031C3D2E203058078400031031
:100C5000000D8000283058078400801F352E20307A
:100C600058078400000801388000283058078400A5
:100C70000310000D8000D80A202EA9237808DA007E
:100C8000DD007E22D90A1B2E5608DD007E22E42ECE
:100C9000A9237808DA00DD007E22D9015908073C33
:100CA000031C772ED8015808073C031C702E2030F7
:100CB000580784000310000C800028305807840077
:100CC000001C682E203058078400000880388000FF
:100CD0002830580784000310000C8000D80A532ED7
:100CE000A9237808DA00DD007E22D90A4E2E5608A4
:100CF000DD007E22E42EA9230310780DDA00DD004A
:100D00007E222B08A3002C08A400A9230310780D31
:100D1000DA00DD007E222A08A2002D08A500A92302
:100D20000310780DDA00DD007E222908A1002E08CC
:100D3000A600A9230310780DDA00DD007E22280822
:100D4000A0002F08A700A9230310780DDA00DD000A
:100D50007E225608DD007E22E42EA9230310780DA2
:100D6000DA00DD007E222808A0002F08A700A923B2
:100D70000310780DDA00DD007E222908A1002E087C
:100D8000A600A9230310780DDA00DD007E222A08D0
:100D9000A2002D08A500A9230310780DDA00DD00BC
:100DA0007E222B08A3002C08A400A9230310780D91
:100DB000DA00DD007E225608DD007E22E42E6A2263
:100DC0005608DD007E22E42E00340A108A140A152B
:100DD0008207AD2E102EE42EE42EE42EE42EDF2E1C
:100DE000E42EE42E152EE42EE42E7B2EE42EE42EAB
:100DF000482EE42EE42E0B2E0130DD007E22780BEF
:100E00002A2F8C2430085A3C03190A2F30087A3CC8
:100E1000031D292F50237808D500550ED600F03039
:100E2000D605242356087804D500A3005508A2004F
:100E30005508A1005508A000D5095508A700550878
:100E4000A6005508A5005508A4000130DD007E224B
:100E50000A2F3B25FC2ED32F5808D900FB217A23DB
:100E60006A223230DD007E22FE226A223230DD002C
:100E70007E222C2F0034D4010130DD007E22780B3D
:100E8000872F8C243B255408D500D7015708D70A53
:100E9000303E84000008D6005508D50AD800031754
:100EA0008D008F010313560803178C0083168C13D3
:100EB0000C15831203130B08F7008B13831603170B
:100EC00055308D00AA308D008C148C18652F0C11B4
:100ED0007708831203138B0456080D3C031D732FF0
:100EE0005508F8007A2FD508031D792F4630D80011
:100EF0002C27462F7808D40030085A3C0319842F39
:100F000030087A3C031D872F5A30D8002C273C2FFD
:100F1000D92FD4015408D500D7015508D50AD800D7
:100F200003178D008F0183168C130C1483120C0889
:100F30000313D600560F9F2F4E30D8002C2757088A
:100F4000D70A303E84005608800056080D3C031D29
:100F5000AC2F5508F800AD2F8D2F7808D4003B2515
:100F600030085A3C0319B82F30087A3C031DB92FBA
:100F7000D4018A2FDB2F84011F30830507308316AD
:100F80009F000510831205140A2B242378080C39BE
:100F9000D300D308031DCE2F102CDB2F5308043CA5
:100FA000031DD42FFC2EDB2F5308083C031DDA2F22
:080FB0003B2FDB2F892F6300AA
:02400E00103967
:00000001FF
